:020000040000FA
:0600000067EF07F012009B
:0600080004EF08F01200F5
:060018000CEF08F01200DD
:0E0020000100FA0E0000E401000002000000E2
:02002E00FC0EC6
:100030008D16961601017E0E006F016BFC0E026F8D
:10004000010E036F846BC769C869C969C66B12006A
:10005000D9CFE6FFE1CFD9FFE652010184511FE17C
:10006000040108BF1BD0400EE66E040EE66E010EC2
:10007000E66E4FEC05F0E552E552E5520101010E46
:10008000846FDF6A400EDF5C09E2DF50EA6A440FEA
:10009000E96E010EEA22EF6ADF2AF4D721D10101CD
:1000A0000451080A01E10BD10F0A01E1D0D0010A85
:1000B00001E1C5D0030A75E0010A61E0070A46E0E4
:1000C000010A01E00DD10101020E446F01013A0E57
:1000D000456F0101010E466F0101010E476F0101DD
:1000E000486B100E496F4A6B4B6B01C14CF102C15A
:1000F0004DF103C14EF1100E01014D5F000E0101E3
:100100004E5B01014F6B0101030E506F0101F80EB0
:10011000516F5269010E536F546B0101080E556FF8
:10012000566B576B586B0101596904010CBF0DD018
:10013000400EE66E440EE66E010EE66E1FEC05F014
:10014000E552E552E5520101846BCAD00101055127
:100150000AE101017F0E006F0101F80E016F0269D3
:10016000010E036F09D001017E0E006F0101016BCA
:10017000FC0E026F010E036F0101846BB1D001010F
:10018000040E856F010100290101855D07E204006D
:10019000ACD8B4EC05F00101852BF4D70101846BD8
:1001A0009FD0E8680101C71905E1E868C81902E1B4
:1001B000E868C91906E105C1C7F106C1C8F107C160
:1001C000C9F1C70EE96E010EEA6EEE500101051984
:1001D00008E1EE500101061904E1EE500101071992
:1001E00000E12AE1DF6A01010951DF5C25E23A0EF4
:1001F0000101D8800955DF24EA6A0A0FE96E010E71
:10020000EA22EF50E66E0101C651EA6A860FE96EF6
:10021000010EEA22E552E750EF6E0101C62B010103
:10022000C72B000EC823000EC9233A0E0101C65D7C
:1002300001E16ED8DF2AD7D70101846B51D068D88D
:100240000101C769C869C9690101846B49D001010D
:10025000070E446F05C145F106C146F107C147F1DC
:1002600008C148F109C149F105C1F6FF06C1F7FF10
:1002700007C1F8FFDF6A01010951DF5C0FE20900E5
:100280003A0E0101D8800955DF24EA6A4A0FE96E67
:10029000010EEA22F5CFEFFFDF2AEDD704010CBFF4
:1002A0000DD0400EE66E440EE66E010EE66E1FECBB
:1002B00005F0E552E552E5520101846B11D06592DB
:1002C000656ADF6AFF0EDF5C09E2E868E85004E077
:1002D000E80600D000D0FAD7DF2AF4D7FF0000D01C
:1002E000E552E552E7CFD9FF1200F66A85C1F7FF64
:1002F000F86AD890F736F836F736F836140EA66E48
:10030000F29E550EA76EAA0EA76EA682A6941200A4
:10031000D9CFE6FFE1CFD9FFE652DF6A0101C6512E
:10032000000832E2C6C100F0016A026A0050010111
:10033000C75DF66E01500101C859F76E0250010108
:10034000C959F86EDF50EA6A860FE96E010EEA229B
:10035000EF50F56E0D00DF2ADF50EA6A860FE96E76
:10036000010EEA22EF50F56E0C00DF2A240EA66E75
:10037000F29E550EA76EAA0EA76EA682020E01016E
:10038000C65D0101C66FCAD7A694E552E552E7CF14
:04039000D9FF12007F
:0C03940064500CE16296040100513C0B27
:1003A000E842E8420D0802E10AD8010C3BD8010CF2
:1003B000040E645C03E1629644D8010C000C73D90E
:1003C000E652040104BF046B0101DC6BD46BD56BF6
:1003D000DA6BDB6B64EC03F0DF6ADF50006E016AFE
:1003E000010E005C000E01581AE20101D55117E11F
:1003F000F76ADF34FE0BF736F66E2D0EF6260E0E7C
:10040000F7220900F5CF00F00800F5CF01F004D085
:1004100001C0FAFF0050F96EFBDFDF2ADED7AFD84C
:10042000E55246D1020E0101D45D09E17CD80401F8
:1004300000BD02D0C80E01D0880E006F1200F8EF88
:1004400002F0040E0101DD5D0CE112C45EFF0F013C
:100450005E51000803E20101050E02D00101030E06
:10046000DD6F0101D40510E111D8020E0101DC5D40
:1004700003E10401840E06D0040104BD02D0C80EBD
:1004800001D0880E046F1200F8EF02F00CD9020EB2
:10049000E1260101080EDA5D000EDB590DE2DAC13A
:1004A000DEFFDBC1DDFFDC5102E1010E03D0DC0524
:1004B00006E1020EDC6F03D0080EDE6EDD6A040179
:1004C00004930491010EDB500413DFCF05F4000EFA
:1004D000DB500101DA5F010EDB50DB5B180ED86FD9
:1004E000040ED96F0101DEA30CD0D6D815E0D6C119
:1004F000F6FFD7C1F7FF0800F550BED8F6E2DB06DD
:10050000F4D7CAD809E0D6C1E9FFD7C1EAFFEF5056
:10051000B3D8F7E2DB06F5D7020EE15C02E2E16A4E
:10052000E552E16EC5D0BFD8020EE126030E0401EC
:100530000015E76E010EE7CFDBFF01C4DFFFDE50E1
:100540000101DA27DD50DB23180ED66F040ED76FBA
:10055000A3D80EE0D6C1E9FFD7C1EAFFEF50D8C15A
:10056000E9FFD9C1EAFFEF6EA7D8F2E2DB06F0D7C8
:10057000020EE15C02E2E16AE552E16E99D0659813
:100580000101D55105E180D8840E006F04011DD012
:10059000040110AF1CD00101DA510401165D010104
:1005A000DB510401175904E216C4DAF117C4DBF178
:1005B0006DDF0101010ED46F67D8800E006F04015A
:1005C000180E066F040E076FC80E046F12000101AB
:1005D000020ED46F0401056BC80E046F0401080EEF
:1005E000016F180E026F040E036FC80E006F120029
:1005F0005AD8E652020E0101D45D35E16550100B68
:1006000032E004010151006E016A080E00182BE16E
:10061000015029E100513C0BE842E8420D0823E17A
:100620000051800B20E1100E026F040E036FDF6A91
:10063000DF50006E016A080E005C000E01581AE2DD
:10064000DF50EA6A180FE96E040EEA22EF50E66EF8
:10065000DF50EA6A100FE96E040EEA22E552E75015
:10066000EF6EDF2AE5D70101D46B0ED88C0E006F38
:100670000401046BE5521CD0D8C1E9FFD9C1EAFFDF
:10068000EF6E01015CEF03F00401080E016F100E24
:10069000026F040E036F1200D9CFE9FFDACFEAFF31
:1006A000EE50ED101200D9CFE6FFE1CFD9FF1200D6
:1006B000E552E7CFD9FF1200D82B000ED923D62B55
:0806C000D723DF06010E120032
:0806C80004011051600BE8422F
:1006D000E842E842E842E842000901E01200115114
:1006E000070A40E00B0A3EE0070A33E0010A23E074
:1006F0000B0A1FE0020A1DE0030A19E0080A10E0D5
:10070000010A0CE00F0A08E0030A01E0120010D908
:100710000101040EDD6F1200B3EF03F0EAEF03F006
:1007200007D90101DF0ED66F010ED76F0CD005EF90
:1007300004F035EF04F000D90101D66FD76BE00E5D
:10074000D627010ED7230101DE930101010EDA6FD6
:100750001200F2D8EA6AE00FE96E010EEA2212C432
:10076000EFFF12001200800E0401105D32E1135100
:10077000030A1FE0010A0AE0030A29E1D9D80101AE
:100780006E0ED66F0D0ED76F120E1ED0B0D8230E80
:10079000F6260E0EBED8020E0101F76AD625F66EB9
:1007A000D751F7220900F5CFDAF10A00F5CFDBF1D6
:1007B0000ED09DD8270EF6260E0EABD8D6C1F6FF6A
:1007C000D7C1F7FF0800F5500101DA6FDB6B0101BB
:1007D000DE831200ADD80F0EE66E4D0EE66E0F0EE4
:1007E000A0D8010EE66EE00EE66E010E9AD812C495
:1007F000DFF10401125104E10101050EDD6F120069
:100800000101060EDD6F09EF05F00401186B196B8D
:10081000040110511F0B020A0DE0030A09E0010A4E
:1008200016E186D80101DEA112D0040118830FD091
:100830007FD80DD050D801E0010E62D8D8C1E9FFB1
:10084000EA6EEF50040B03E00401010E186F010182
:10085000D5050AE10101180ED66F040ED76F01010C
:10086000DE930101020EDA6F1200040112050EE19F
:1008700010511F0B00090AE15BD8030E0401115D42
:1008800003E10101DE8102D00101DE910401125178
:1008900021E110511F0B02081DE114510F0B00093B
:1008A00019E019D801E0010E2BD8030E0401115DE7
:1008B00002E1840E03D014AF07D0400ED8C1E9FF87
:1008C000D9C1EAFFEF6E1200880ED8C1E9FFD9C185
:1008D000EAFFEF6E120030D80F0B080DF350016ADB
:1008E000000F006E040E01221451800B120020D85C
:1008F00004011251F66EF76AD890F636F7361200F8
:10090000040DF35001010024D86F000E0120D96FAF
:100910001200F7220900F5CFD6F10A00F5CFD7F182
:100920001200E66E40EC06F0E552E552E552120088
:100930000101010ED56F1200FBDF040114511200FA
:10094000040110511F0B010801E01200145101E0D5
:100950001200060E115D24E11351230A1FE0010A63
:100960000DE0030A1BE1DCD80101DF0505E101010F
:10097000920ED66F0D0ED76F090E0DD0D1D8010192
:10098000DF0505E10101070ED66F0E0ED76F0101DD
:10099000DF0504E11C0E0101DA6FDB6B0101DE8370
:1009A00004011051600BE842E842E842E842E842A4
:1009B000010801E0120011510B0A25E0080A17E0B6
:1009C000090A11E0080A09E00B0A05E0080A01E03B
:1009D000120007EF05F008EF05F0A2D80101E10EC3
:1009E000D66F010E09D09CD813C4E1F1120098D83B
:1009F0000101E20ED66F010ED76F0101DE930101F6
:100A0000010EDA6F12008CD812C4E2F1120012004B
:100A100012000101E36B0F011E0E4D6F0401400E29
:100A2000096F200E0A6F040E0B6F880E086F040109
:100A3000600E0E6F040E0F6F400E0C6F1200D9CFB8
:100A4000E6FFE1CFD9FFE652FC0EDB50400805E29D
:100A5000400EF36EFC0EF3CFDBFFDF6AFC0EDB50C3
:100A6000DF5C0FE2DF5050D8EF50E66EDF50EA6AED
:100A7000600FE96E040EEA22E552E750EF6EDF2ABE
:100A8000EDD7FC0EDBCF0DF4400E04010C170C7DEE
:100A9000880E0C13E552E552E7CFD9FF1200D9CFEB
:100AA000E6FFE1CFD9FF0101E36B040108BF26D0C7
:100AB000FC0EDBCF00F00951D880005403E2FC0E9D
:100AC00009C4DBFF0101E36BFC0EDB50E35D0FE2C9
:100AD000E351EA6A200FE96E040EEA22EF50E66E57
:100AE000E35112D8E552E750EF6EE32BEDD7040146
:100AF000400E096F0817087D880E08130101E351A5
:100B0000E552E7CFD9FF1200E76EFD0EDBCFE9FF1C
:100B1000FE0EDBCFEAFFE750E926000EEA221200C4
:080B20000101020ED56F120065
:080B280065A60ED80101DD05F0
:100B30000AE165BA08D0626A0F015C6B5C815C896E
:100B40000101020EDD6F1200656A0F015C6B6586A4
:100B50000101010EDD6F1200656A0F015C6B01017E
:100B6000DD6B1200ACEF05F00101DD5101E1120077
:100B70006250040B05E00F015C51040B01E03DD80D
:100B800065B212006250010B05E00F015C51010BD0
:100B900001E04DD86250100B05E00F015C51100BC5
:100BA00001E022D86250200B05E00F015C51200BC0
:100BB00001E02BD8030E0101DD5D01E2120001010D
:100BC000E66B040EE65D0FE26250080B0CE00F01CD
:100BD0005C51080B08E0CAEC01F0000901E16296E3
:100BE0000101E62BEED712000F015C856298658249
:100BF000A198A0880300A098120065920F015C954F
:100C000062A402D06294FCD712000F014CA10DD057
:100C1000800E0401005D07E1840E0401045D03E120
:100C200004018C0E006F0F014C91629A1200636AEE
:100C3000626A0F019F0E5D6F0F017B0E5C6F0F01EB
:100C40005E6B0F0EE66E4D0EE66E0F0EE66E18D85A
:100C5000E552E552E5520F01160E4C6F62A605D023
:100C6000629600D000D00000F9D76598F8EC02F049
:100C70000101DE910101DF6B0101030EDD6F120046
:100C8000D9CFE6FFE1CFD9FFFD0EDBCFE9FFFE0EA6
:100C9000DBCFEAFFFC0EDB5004E0EE6AFC0EDB0665
:0A0CA000F9D7E552E7CFD9FF1200A3
:060CAA0081A802D000EF5A
:100CB00008F00ED8040037D83AD8060E0101DD5DE1
:100CC00005E16550020B02E128EC00F0F3D71200B9
:100CD000D9CFE6FFE1CFD9FF020EE126580EDE6E36
:100CE000020EDD6E9B8CDFCF00F0DF06010EDBCF46
:100CF00001F001E2DB0600500110F5E10F01140ED6
:100D00005F6F0101DD6B0101DE6B0101DF6B17EC31
:100D100000F0020EE15C02E2E16AE552E16EE552AA
:100D2000E7CFD9FF120094EC05F0B4EF05F0010114
:100D3000E451E51104E1100EE46F270EE56FE407BE
:100D4000000EE55B060E0101DD5D02E28D828D90F5
:100D5000060EDD5D0BE10101E451E51107E18D7245
:0E0D60008D50020B02E08D9012008D8012006B
:020D6E00120170
:100D7000000200000008D8043C000200010200014B
:100D800009022900010100C0320904000002030029
:100D90000000092111010001221C00070581034008
:100DA0000001070501034000010403090434034D59
:100DB000006900630072006F0063006800690070E2
:100DC00000200054006500630068006E006F006C36
:100DD000006F0067007900200049006E0063002E5C
:100DE00000260348004900440020005500530042FB
:100DF00000200042006F006F0074006C006F006103
:100E00000064006500720006FFFF0901A1011901DD
:100E10002940150025FF75089540810219012940D8
:0F0E20009102C0800D800DA90DAD0DE10D4009AF
:100E3000200EF66E000EF76E000EF86E010109002E
:100E4000F550CF6F0900F550D06F03E1CF6701D0A7
:100E50003DD00900F550CA6F0900F550CB6F09006D
:100E6000F550CC6F09000900F550E96E0900F55006
:100E7000EA6E090009000900F550CD6F0900F55030
:100E8000CE6F09000900F6CFD1F1F7CFD2F1F8CF3C
:100E9000D3F1CAC1F6FFCBC1F7FFCCC1F8FF010106
:100EA000CD5302E1CE5307E00900F550EE6ECD07B9
:100EB000F8E2CE07F9D7D1C1F6FFD2C1F7FFD3C10F
:0E0EC000F8FF0101CF07000ED05BBFD7120074
:020ECE001EEE16
:100ED00000F02EEE00F0F86A049C18EC07F07CECB1
:0A0EE00007F055EC06F0FBD71200F6
:060EEA0000EE00F00F0E07
:080EF000EE6AEA62FDD7120070
:020EF8001200E6
:020EFA000000F6
:020000040001F9
:01FFF800AA5E
:01FFF900F710
:01FFFA000501
:01FFFB00FF06
:01FFFC00F014
:01FFFD00F70C
:00000001FF
